:1000000012C02CC02BC02AC029C028C027C026C0BF
:1000100025C078C123C033C054C020C01FC01EC03B
:100020001DC01CC01BC011241FBECFE5D4E0DEBF25
:10003000CDBF12E0A0E6B0E0EAE0F5E102C0059035
:100040000D92A43AB107D9F713E0A4EAB2E001C0D7
:100050001D92A931B107E1F7E6D455CAD1CF90BDC1
:1000600089B988E18AB986E880BD1092A70210920A
:10007000A6021092E9021092E802579A08951F9280
:100080000F920FB60F9211242F938F939F93EF939C
:10009000FF939CB18091A6028F5F81708093A6022E
:1000A0002091A702E4EAF2E0E80FF11D9083FF91AE
:1000B000EF919F918F912F910F900FBE0F901F90F6
:1000C00018951F920F920FB60F9211248F939F9342
:1000D000EF93FF939091E8028091E902981761F005
:1000E000E091E902EF5FEF73E093E902F0E0E85599
:1000F000FD4F80818CB901C05598FF91EF919F9180
:100100008F910F900FBE0F901F9018959091A6029F
:100110008091A70220E0981321E0822F089590910A
:10012000A6028091A7029817D1F3E091A702EF5F92
:10013000E170E093A702F0E0EC55FD4F8081089557
:10014000282F9091E8029F5F9F738091E902981792
:10015000E1F3E92FF0E0E855FD4F20839093E802AA
:10016000559A08951F93CF93DF93EC0197FF08C032
:100170008DE2E6DFD095C195DF4F02C0C051D74276
:1001800027E2C031D207D4F702C0C85ED34033E0C3
:10019000C83ED307D4F790E002C0C456D040892FA0
:1001A0009F5FC436D105CCF790E001C02A97192F84
:1001B0009F5FCA30D105D4F7805DC2DF812F805D9B
:1001C000BFDF9E01205D822FBBDFDF91CF911F91AA
:1001D0000895EF92FF920F931F93CF93DF93EC015B
:1001E00097FD02C090E004C0D095C195DF4F9FEF0E
:1001F00080E002C0C051D742E82E8F5F27E2C031B5
:10020000D207C4F780E002C0C85ED340F82E8F5FEB
:1002100033E0C83ED307C4F780E002C0C456D040E4
:10022000082F8F5FC436D105CCF780E001C02A9734
:10023000182F8F5FCA30D105D4F7992311F08DE2C2
:1002400001C080E27DDF8E2D805D7ADF8F2D805DA5
:1002500077DF802F805D74DF812F805D71DF9E01ED
:10026000205D822F6DDFDF91CF911F910F91FF9065
:10027000EF9008951F93CF93DF93182FC0E0D0E045
:10028000812F881F8827881F805D5ADF2196C830FC
:10029000D10511F0110FF4CFDF91CF911F91089587
:1002A0000F931F93182F882311F020E003C080E3E1
:1002B00019C01456322F2F5F812F90E0843691059C
:1002C000C4F720E001C01A50022F2F5F812F90E069
:1002D0000A97CCF7832F805D33DF802F805D30DF7E
:1002E000812F805D2DDF1F910F910895CF93DF93B4
:1002F000EC0102C025DF219688818823D9F7DF91A0
:10030000CF9108951F920F920FB60F9211245F9311
:100310006F937F938F939F93AF93BF9380911603B7
:100320009091170301969093170380931603809181
:1003300016039091170362E370E09AD8892B19F4A1
:1003400081E080931803BF91AF919F918F917F912E
:100350006F915F910F900FBE0F901F9018951092A4
:100360001703109216031092180383B7836083BF9C
:1003700012BE89B7816089BF089589B78E7F89BF12
:10038000109217031092160389B7816089BF0895F0
:1003900089B7816089BF089589B78E7F89BF089525
:1003A000E199FECF9FBB8EBB6DBBF894E29AE19AB8
:1003B00078940895E199FECF9FBB8EBBE09A8DB3F0
:1003C0000895EAEEF2E080E991E08193919322E0D2
:1003D000EA3FF207D1F786E086B983E487B9379A16
:1003E000369A0895369921C047B14770E42FF0E05E
:1003F00064B175B1EE0FFF1FE651FD4F20813181D1
:10040000C901880F991F820F931F860F971F96951A
:10041000879596958795918380834F5F483009F43F
:1004200043E04770406447B9369A0895883018F021
:10043000E0E0F0E009C0E82FF0E0EE0FFF1FE6512A
:10044000FD4F0190F081E02DCF010895382F6623F4
:1004500061F422B381E090E002C0880F991F3A95C1
:10046000E2F78095822382BB089522B381E090E079
:1004700002C0880F991F3A95E2F7282B22BB0895F6
:100480008F929F92AF92BF92CF92DF92EF92FF92A4
:100490000F931F93CF93DF934B0100917501109140
:1004A0007601EC01081719070CF4E801A09073011C
:1004B000B0907401BE01882777FD8095982F91D563
:1004C0006B017C011C161D0634F4B801882777FDEA
:1004D0008095982F05C0B501882777FD8095982FC6
:1004E00080D59B01AC01C701B601D6D47B018C013C
:1004F000B401882777FD8095982F73D59B01AC01B7
:10050000C801B701D4D3C7D5CB01DF91CF911F91DB
:100510000F91FF90EF90DF90CF90BF90AF909F90A2
:100520008F900895CF93DF93EC0127DF809116031E
:10053000909117038C179D07C8F31FDFDF91CF91B0
:100540000895CF93DF93EC012091160330911703A8
:10055000999B03C08AEF90E002C084E690E0821786
:10056000930778F40ADF8881882329F4929881E040
:100570008883939A06C0929A809100038111939880
:100580001882DF91CF9108951F93182F80E690E095
:10059000ADDE812F805DD4DD80E2D2DD1F91089534
:1005A000EF92FF921F93CF93DF937C01EB0110E05A
:1005B000812FEADF83E690E099DE209719F487E641
:1005C00090E00FC08DE690E091DECE018FDEC70196
:1005D000C9DD82E790E08ADE812F805DB1DD84E7AE
:1005E00090E084DE1F5F163019F7DF91CF911F91E5
:1005F000FF90EF900895EF92FF920F931F93CF9388
:10060000DF93062F7A01E901182F15C0812FBCDF77
:1006100083E690E06BDE209719F487E690E009C04E
:100620008DE690E063DECE0161DEC7019BDD84E7ED
:1006300090E05CDE1F5F10174CF3DF91CF911F91AC
:100640000F91FF90EF900895FF920F931F93162F35
:10065000F42E022F99DF8BE790E048DE1F3F19F060
:10066000812F805D6DDD8F2D6BDD0F3F11F0802FB1
:1006700017DE8EE790E03ADE1F910F91FF9008950C
:10068000EF92FF920F931F93E82E989903C010E00A
:1006900006E004C010910503012F0F5F8E2D809599
:1006A0008623F82E81FF13C0E2FC09C0809102036B
:1006B0008F5F80930203803110F01092020340910B
:1006C000020321E830E050E0602F812F94DFF0FE3C
:1006D0000CC0E2FC02C0109203034091030323E824
:1006E00030E050E0602F812F86DFF3FE30C0E2FC67
:1006F0000DC020E046E56FEF80910503A5DF2FEFE9
:1007000046E46FEF809105039FDF21C0989918C0E0
:100710008091040380FF05C060E070E080E090E01D
:1007200004C065E870E0869590E03ADF80910403AC
:100730008F5F80930403803150F01092040307C050
:1007400020E030E040E050E0602F812F54DFF5FEE4
:100750001EC08091050318DF8AE890E0C7DD809114
:10076000050312DF81E990E0C1DD809105030CDF14
:1007700088E990E0BBDD22E344E56FEF809105035B
:1007800063DF2FEF43E46FEF809105035DDFF4FE3D
:1007900020C080910503F8DE82EA90E0A7DD8E2D6F
:1007A00090E0809590958C7090708830910541F024
:1007B0008C30910541F0049749F489EA90E008C033
:1007C0008DEA90E005C081EB90E002C085EB90E0FF
:1007D0008DDD1F910F91FF90EF900895FF920F9381
:1007E0001F93CF93DF93F82E062FEA01122F2F3F8E
:1007F00009F41EEF8F2DC8DE8BE790E077DD0F3F09
:1008000019F0802F805D9CDC88E49ADCCE01AADCA4
:100810008EE790E06BDD212F46E5602F8F2D14DFF2
:100820002FEF46E4602F8F2D0FDFDF91CF911F91C7
:100830000F91FF9008951F93CF93DF93EC01CB01AD
:1008400064E170E01DDE2091FA023091FB02280F76
:10085000391F3093FB022093FA0281E029363807D2
:1008600034F0285631403093FB022093FA028091F5
:10087000FA029091FB0297FF06C088599E4F909311
:10088000FB028093FA0261EF7FEFCE01F9DD209148
:1008900077012091FC023091FD02280F391F30931F
:1008A000FD022093FC022E3F310534F08EEF90E0E4
:1008B0009093FD028093FC028091FC029091FD02D6
:1008C000029724F41092FD021092FC0298990EC037
:1008D00010E04091FA025091FB022091FC026FEF70
:1008E000812F7CDF1F5F1630A1F70AC04091FA020A
:1008F0005091FB022091FC026FEF809105036EDFA7
:10090000DF91CF911F910895FF920F931F93CF9383
:10091000DF93082F162FF42E22E344E595DECF2D2A
:10092000D0E0FE01E858FE4F208142E5612F802F84
:100930008BDEFE01E058FE4F208147E4612F802FBF
:1009400083DEC857DE4F288142E4612F802F7CDE92
:100950002FEF46E4612F802F77DEDF91CF911F913B
:100960000F91FF9008951F9380EC87BB8FE388BBA6
:1009700014BA87E085BB8EE081BB80EF82BB8BE041
:1009800090E06DDB1EDDEBDC789480B390E0809529
:100990009095807F907024E0959587952A95E1F752
:1009A0008F70809305032CE38202900111242C5E4A
:1009B0003F4F3093FB022093FA028FE790E0909331
:1009C000FD028093FC0289EB90E090DC2091FA021A
:1009D00048E46FEF8091050337DE2091FC0246E585
:1009E0006FEF8091050330DE2FEF46E46FEF8091CB
:1009F00005032ADE10E009C0939884E690E092DDBA
:100A0000939A84E690E08EDD1F5F212F30E0809185
:100A10000503992787FD9095281739076CF3939A5A
:100A2000929A1F9108957F928F929F92AF92BF9258
:100A3000CF92DF92EF92FF920F931F93DF93CF93AA
:100A40000F92CDB7DEB719828EDF56E0C52E53E088
:100A5000D52EF6011192119223E0E631F207D1F77B
:100A6000AA24BB2420C0BEDC0F5F1F4F3FE100342F
:100A70001307C9F7F70100811181892DD7DC080F11
:100A8000191FF701019311937F019394F8E09F16CA
:100A900019F000E010E0E7CF0894A11CB11C28E099
:100AA000A216B10431F046E0E42E43E0F42E99247E
:100AB000F0CFF6018081918133E0969587953A9544
:100AC000E1F7819391936F01F6E1CF16F3E0DF0632
:100AD00081F74E010894811C911C7724739482DC69
:100AE000C4012FDD809118038823C9F310921803E5
:100AF00083E09CDC895D93401CF07092000302C08F
:100B00001092000385E092DC2091100330911103D4
:100B10005C01A21AB30A8091920190919301F501B0
:100B2000E81BF90BCF01F7FF03C0909581959F4F0C
:100B300006970CF18091050327DD87EC90E0D6DB6A
:100B40009501B7FE04C0222733272A193B0980915B
:100B5000900190919101281739071CF480E3F0DA95
:100B600007C060916D0170916E01C50189DCFADAF0
:100B70008AEC90E0BBDBB0929301A092920184E0FA
:100B800055DC20910E0330910F038C01021B130BD7
:100B900080919401909195019801281B390BC9010E
:100BA00037FF03C0909581959F4F069784F1809100
:100BB0000503EADC80ED90E099DB980117FF04C0A3
:100BC00022273327201B310B8091900190919101B6
:100BD000281739071CF480E3B3DA16C099990AC0C4
:100BE0006091710170917201709561957F4FC8019C
:100BF00047DC09C060916F0170917001709561953B
:100C00007F4FC8013DDCAEDA8AEC90E06FDB1093D9
:100C100095010093940186E009DC20911203309144
:100C200013036C01C21AD30A87E000DC209114037D
:100C3000309115037C01E21AF30A80917701882331
:100C4000A1F083ED90E052DBC8018CDA88ED90E0F2
:100C50004DDBC50187DA8CED90E048DBC60182DA16
:100C600080EE90E043DBC7017DDAC601D7FE04C009
:100C7000882799278C199D090B974CF4C701F7FE1B
:100C800004C0882799278E199F090B971CF0B6017D
:100C9000C701D1DD16B360919A01161711F0812FAB
:100CA000EFDC10939A0183B38091770118CFA0E213
:100CB000B0E0ECE5F6E0F0C369837A838B839C8334
:100CC0002D833E834F835887BE01675F7F4FCE01E0
:100CD000019656D3BE016F5E7F4FCE01059650D36D
:100CE0009985923088F089898230C8F0943019F45F
:100CF000823051F404C0843029F4923081F48BE9BD
:100D000091E0C6C0923049F420E09A858A89981310
:100D100021E02A87CE010996BBC0823049F420E049
:100D20009A858A89981321E02A8BCE014196B0C01A
:100D30002D843E844F8458886D887E888F88988C57
:100D4000EE24FF248701AA24BB24650140E050E083
:100D500060E070E0E0E0F0E0C10181709070892B0C
:100D6000E9F0E60CF71C081D191D9A01AB012A0DCC
:100D70003B1D4C1D5D1D80E090E0A0E0B0E0E6145E
:100D8000F7040805190520F481E090E0A0E0B0E048
:100D9000BA01A901480F591F6A1F7B1FAA0CBB1C6F
:100DA000CC1CDD1C97FE08C081E090E0A0E0B0E024
:100DB000A82AB92ACA2ADB2A3196E032F10549F07D
:100DC000660C771C881C991C56944794379427947A
:100DD000C3CFFA85EA892B893C898B859C85280FAE
:100DE000391F2E5F3F4F17C0CA0181709070892B49
:100DF00061F016950795F794E79480E090E0A0E005
:100E0000B0E8E82AF92A0A2B1B2B769567955795A7
:100E100047952F5F3F4F77FDE7CF0CC0440F551F1D
:100E2000661F771F17FD4160EE0CFF1C001F111F8E
:100E300021503040403090E0590790E0690790E43D
:100E4000790760F32B8F3C8FDB01CA018F7790709D
:100E5000A070B07080349105A105B10561F447FD23
:100E60000AC0E114F1040105110529F0405C5F4F4F
:100E70006F4F7F4F40781A8EFE1711F081E08A8FF6
:100E80004D8F5E8F6F8F78A383E0898FCE01499657
:100E9000A2D1A096E2E11CC3A8E1B0E0E1E5F7E051
:100EA00003C369837A838B839C832D833E834F8323
:100EB0005887B9E0EB2EF12CEC0EFD1EB701CE01E8
:100EC00001965ED28E010F5E1F4FB801CE010596CE
:100ED00057D22985223008F47CC03989323010F489
:100EE000B8017AC08A859A8989278A87243011F0C7
:100EF000223031F4231709F06CC06BE971E06CC04B
:100F0000343039F41D861E861F86188A1C861B867F
:100F100004C0323021F484E08987B7015DC02B859D
:100F20003C858B899C89281B390B3C872B87ED845A
:100F3000FE840F851889AD88BE88CF88D88CEA14C6
:100F4000FB040C051D0540F4EE0CFF1C001F111FD7
:100F5000215030403C872B8720E030E040E050E0DB
:100F600080E090E0A0E0B0E46FE170E0EA14FB0400
:100F70000C051D0540F0282B392B4A2B5B2BEA185A
:100F8000FB080C091D09B695A79597958795EE0C5A
:100F9000FF1C001F111F6150704041F7DA01C901A9
:100FA0008F779070A070B07080349105A105B10565
:100FB00061F427FD0AC0E114F1040105110529F0CF
:100FC000205C3F4F4F4F5F4F20782D873E874F87E4
:100FD000588BBE01675F7F4FCB01FDD06896EAE07A
:100FE0007FC2A8E0B0E0E6EFF7E05FC29B01AC0192
:100FF00083E08983DA01C9018827B7FD83959927A2
:10100000AA27BB27B82E211531054105510519F432
:1010100082E0898339C08823A9F0203080E0380736
:1010200080E0480780E8580729F460E070E080E03D
:101030009FEC2EC0EE24FF248701E21AF30A040B72
:10104000150B02C079018A018EE1C82ED12CDC82F9
:10105000CB82ED82FE820F831887C801B7016CD066
:1010600001971816190684F4082E04C0EE0CFF1C14
:10107000001F111F0A94D2F7ED82FE820F8318879A
:10108000C81AD90ADC82CB82BA82CE010196A3D0DB
:101090002896E9E026C2ACE0B0E0E0E5F8E00CC25A
:1010A00069837A838B839C83BE016B5F7F4FCE0104
:1010B000019666D18D81823061F1823050F18430A9
:1010C00021F48E81882351F12EC02F81388537FD80
:1010D00020C06E812F3131051CF06623F9F023C04A
:1010E0008EE190E0821B930B29853A854B855C85C8
:1010F00004C056954795379527958A95D2F766236C
:10110000B1F050954095309521953F4F4F4F5F4F2F
:101110000EC020E030E040E050E009C02FEF3FEF8C
:101120004FEF5FE704C020E030E040E050E8B90155
:10113000CA012C96E2E0DCC1EF92FF920F931F935D
:101140007B018C0180E0E81680E0F80681E008076A
:1011500080E0180788F48FEFE816F1040105110507
:1011600031F028F088E090E0A0E0B0E017C080E027
:1011700090E0A0E0B0E012C080E0E81680E0F80661
:1011800080E0080781E0180728F088E190E0A0E0FF
:10119000B0E004C080E190E0A0E0B0E020E230E008
:1011A00040E050E0281B390B4A0B5B0B04C016953E
:1011B0000795F794E7948A95D2F7F701ED55FE4F1E
:1011C0008081281B310941095109C9011F910F91E3
:1011D000FF90EF900895DF92EF92FF920F931F938D
:1011E000FC01E480F58006811781D1808081823006
:1011F00048F480E090E0A0E1B0E0E82AF92A0A2B68
:101200001B2BA5C0843009F49FC0823021F4EE244A
:10121000FF24870105C0E114F1040105110519F44B
:10122000E0E0F0E096C0628173819FEF6238790759
:101230000CF05BC022E83FEF261B370B2A3131054B
:101240002CF020E030E040E050E02AC0B801A701D7
:10125000022E04C076956795579547950A94D2F764
:1012600081E090E0A0E0B0E004C0880F991FAA1FC1
:10127000BB1F2A95D2F70197A109B1098E219F21A1
:10128000A023B1230097A105B10521F081E090E0F2
:10129000A0E0B0E09A01AB01282B392B4A2B5B2B45
:1012A000DA01C9018F779070A070B0708034910519
:1012B000A105B10539F427FF09C0205C3F4F4F4F0E
:1012C0005F4F04C0215C3F4F4F4F5F4FE0E0F0E0C5
:1012D0002030A0E03A07A0E04A07A0E45A0710F047
:1012E000E1E0F0E079018A0127C06038710564F51A
:1012F000FB01E158FF4FD801C7018F779070A070B4
:10130000B07080349105A105B10539F4E7FE0DC038
:1013100080E490E0A0E0B0E004C08FE390E0A0E0C3
:10132000B0E0E80EF91E0A1F1B1F17FF05C0169537
:101330000795F794E794319687E016950795F7940B
:10134000E7948A95D1F705C0EE24FF248701EFEFDB
:10135000F0E06E2F679566276795902F9F77D7945B
:10136000DD24D7948E2F8695492F462B582F5D2943
:10137000B701CA011F910F91FF90EF90DF90089580
:10138000FC01DB01408151812281622F6F7770E087
:10139000221F2227221F9381892F880F822B282F1B
:1013A00030E0991F9927991F11969C931197211549
:1013B0003105A9F5411551056105710511F482E06A
:1013C00037C082E89FEF13969C938E9312979A01F1
:1013D000AB0167E0220F331F441F551F6A95D1F7F9
:1013E00083E08C930DC0220F331F441F551F1296AC
:1013F0008D919C911397019713969C938E931297BE
:10140000203080E0380780E0480780E4580758F330
:1014100014962D933D934D935C93179708952F3F0A
:10142000310579F4411551056105710519F484E020
:101430008C93089564FF03C081E08C9312C01C92CA
:1014400010C02F57304013963C932E93129783E091
:101450008C9387E0440F551F661F771F8A95D1F73D
:10146000706414964D935D936D937C9317970895D4
:10147000AA1BBB1B51E107C0AA1FBB1FA617B707BA
:1014800010F0A61BB70B881F991F5A95A9F78095D6
:101490009095BC01CD0108952F923F924F925F929B
:1014A0006F927F928F929F92AF92BF92CF92DF9274
:1014B000EF92FF920F931F93CF93DF93CDB7DEB7D9
:1014C000CA1BDB0B0FB6F894DEBF0FBECDBF09946D
:1014D0002A88398848885F846E847D848C849B84C4
:1014E000AA84B984C884DF80EE80FD800C811B81D2
:1014F000AA81B981CE0FD11D0FB6F894DEBF0FBE01
:0A150000CDBFED010895F894FFCF70
:10150A007B36003C4D20005653543E7D00565046D3
:10151A0020005F002E6D70333E7D003C4C003E7D06
:10152A000068006100736F6E6700247030302A7D96
:10153A0000247330302A7D005B48414C5420305DD2
:10154A007D005B4D4F44452000315D7D00325D7D5D
:10155A0000335D7D00305D7D0052656D6F746520DE
:10156A0076312E330D0A002473002A7D0A0D2000DD
:10157A002470000A0D443A0020533A0020483A00E9
:10158A0020563A000C0030303230383037320030D2
:10159A003036383137323700303233353534383235
:1015AA000030353132363034350030363937333061
:1015BA003837003133353334383531003337353540
:1015CA00383538003131393039323932003037382C
:1015DA00363336323100303838353737383800301C
:1015EA0039393339393638003139393836333834BC
:1015FA00000000E600EF00F80001010A0113011CD7
:10160A000124012D0136013F0148015101640046C0
:10161A00006400F401F40101FE0000FEFE00FE0079
:10162A0000FE0000FEFEFE000000FEFE00FEFE00C0
:10163A0003009CFF9CFF9CFF9CFFFF000000000032
:10164A00000000000102020303030304040404046B
:10165A000404040505050505050505050505050533
:10166A000505050606060606060606060606060613
:10167A000606060606060606060606060606060600
:10168A0006060607070707070707070707070707E3
:10169A0007070707070707070707070707070707D0
:1016AA0007070707070707070707070707070707C0
:1016BA0007070707070707070707070707070707B0
:1016CA000707070808080808080808080808080893
:1016DA000808080808080808080808080808080880
:1016EA000808080808080808080808080808080870
:1016FA000808080808080808080808080808080860
:10170A00080808080808080808080808080808084F
:10171A00080808080808080808080808080808083F
:10172A00080808080808080808080808080808082F
:10173A00080808080808080808080808080808081F
:04174A000808080083
:00000001FF
